:100000000C9478020C9495020C9495020C94950231
:100010000C9495020C9495020C9495020C94950204
:100020000C9495020C9495020C94491F0C941B207F
:100030000C943B1A0C9495020C9495020C94950226
:100040000C9495020C9495020C9495020C949502D4
:100050000C9495020C94C31A0C9495020C9495027E
:100060000C9495020C9495020C9495020C949502B4
:100070000C9495020C9495020C9495020C949502A4
:100080000C9495020C9495020C9495020C94950294
:100090000C9495020C9495020C9495020C94950284
:1000A0000C9495020C9495020C949502A502AA0258
:1000B000B102D402B602B802CB02F6022D062D061A
:1000C00059065906C106DF06F707F707EA06830750
:1000D000940794078820AF20A721AF20A721FB20F9
:1000E0001E21A721752184212B0014001A0008006D
:1000F000150017001C0018000C00120013002A0045
:10010000290004001600070009000A000B000D007A
:100110000E000F0033003400E1001D001B0006003C
:1001200019000500110010003600370038002800C3
:10013000AD5DE000E200E300AB5D2C002C00AC5DA7
:100140005000510052004F002B0014001A0009000B
:1001500013000A000D000F0018001C0033002A00D5
:100160002900040015001600170007000B001100FD
:1001700008000C0012003400E1001D001B00060006
:10018000190005000E001000360037003800280066
:10019000AD5DE000E200E300AB5D2C002C00AC5D47
:1001A0005000510052004F002B0034003600370041
:1001B00013001C0009000A00060015000F002A00A9
:1001C000290004001200080018000C0007000B00B2
:1001D0001700110016003800E100330014000D0074
:1001E0000E001B00050010001A0019001D00280059
:1001F000AD5DE000E200E300AB5D2C002C00AC5DE7
:100200005000510052004F0035021E021F02200212
:1002100021022202230224022502260227022A00AA
:100220004C003A003B003C003D003E003F002D02E8
:100230002E022F0230023102010040004100420034
:10024000430044004500320264024A004D000100B0
:100250000100010001000100010001000100010096
:10026000AB00AA00A900AE0035001E001F00200050
:1002700021002200230024002500260027002A0058
:100280004C003A003B003C003D003E003F002D008A
:100290002E002F00300031000100400041004200DC
:1002A000430044004500320064004B004E00010052
:1002B0000100010001000100010001000100010036
:1002C000AB00AA00A900AE001E001E001E001E000A
:1002D0001E001E001E001E001E001E001E001E002E
:1002E000000014001A000800150017001C00180078
:1002F0000C00120013002F0000000400160007007D
:1003000009000A000B000D000E000F00330034003E
:10031000AE5D0000000006001900000000001100A2
:1003200010000000000000000100005C015CC35CE4
:10033000C45CC65CC75CC85CC95CCA5CCB5C4C0076
:1003400001000100295C1D5C1E5C135C0A5CA75D5A
:10035000A85DA95DAA5D010001002B5C2A5C265CFA
:10036000275C2C5C2D5C00000000010001000100F6
:100370000100010001000100010001000100010075
:1003800001000100010001000E0343006F006E0038
:1003900074007200610000000E03430061007200EF
:1003A000740065006C0000000403090409023B00AE
:1003B000020100A0FA090400000103010100092163
:1003C0001101000122400007058103080001090412
:1003D0000100010300000009211101000122B60003
:1003E00007058203200001120100020000000854EA
:1003F00043010001000102000105010902A101857C
:10040000020901A100050919012908150025019516
:1004100008750181020501093009311581257F9593
:10042000027508810609381581257F9501750881B7
:1004300006050C0A38021581257F9501750881068D
:10044000C0C005010980A101850319012AB7001563
:100450000126B700950175108100C0050C0901A1A6
:1004600001850419012AA002150126A00295017533
:10047000108100C005010906A1018506050719E0E4
:1004800029E7150025019508750181020507190066
:1004900029EF1500250195F0750181020508190164
:1004A0002905950575019102950175039101C00516
:1004B000010906A101050719E029E71500250195A5
:1004C0000875018102950175088101050719002948
:1004D000FF150026FF009506750881000508190123
:1004E0002905950575019102950175039101C000DB
:1004F00011241FBECFEFDAE0DEBFCDBF11E0A0E0D8
:10050000B1E0E4EBF4E402C005900D92AC38B10721
:10051000D9F722E0ACE8B1E001C01D92A73AB207DA
:10052000E1F70E9404140C9458220C940000CF931D
:10053000875A9D458830910508F05FC0FB018A5AB3
:100540009F4FC281FC010C94EF21CC2309F456C0CB
:1005500080E004C0CC2309F451C081E00E94510323
:100560004AC0CC2309F44AC082E0F8CF83E001C03E
:1005700084E0CC2341F00E943F0946E064E083E040
:100580000E94BF0338C00E94600946E064E083E037
:100590000E94BF0333C085EECC2319F00E94B20441
:1005A0002AC00E945C052AC0CC2341F184E00E944D
:1005B000600983E00E94600986E00E94600985E08E
:1005C0000E943F090E94C30E811102C00E94700F59
:1005D0000E94DB0E90938502806880938402809154
:1005E0008402909185020E94EC0E05C0CC2331F06C
:1005F00085E00E946009C0E001C0C1E08C2FCF916E
:10060000089581E008950C94970208950C940503D1
:100610001F93CF93DF9300D000D01F92CDB7DEB7EA
:1006200049835A836B8330918F0189819A8131117B
:1006300014C0662359F0222349F00E94340A182F6F
:10064000682F89819A810E94DD0903C00E94080AEF
:10065000182F69817A81812F04C00E94340A698130
:100660007A810F900F900F900F900F90DF91CF91A4
:100670001F910C946F11FC01262F408151816281E2
:10068000738184810C94080381E00895CF93DF93F4
:10069000EC0160E00E943B03BE01DF91CF910C941E
:1006A0000603CF92DF92EF92FF92C12CD12C7601FC
:1006B000C39404C0CC0CDD1CEE1CFF1C8A95D2F741
:1006C0008C2D0E94D60EC701B601FF90EF90DF90EF
:1006D000CF900C94DF088F929F92AF92BF92CF92EF
:1006E000DF92EF92FF920F931F936B017C0181E0E9
:1006F00090E0A0E0B0E04C015D0104C0880C991CC2
:10070000AA1CBB1C4A95D2F7AC01BD0104C0440F22
:10071000551F661F771F2A95D2F7482959296A293C
:100720007B2904C0880F991FAA1FBB1F0A95D2F707
:100730008A019B010C211D212E213F2140175107C9
:100740006207730739F4BC01CD016C297D298E291C
:100750009F290AC080959095A095B095BC01CD01C8
:100760006C217D218E219F211F910F91FF90EF9091
:10077000DF90CF90BF90AF909F908F9008950F9390
:10078000382F262F6091AE017091AF018091B0019A
:100790009091B101042F432F0E946B030F910C9491
:1007A00019090C94B5120C94B11208950E9487088F
:1007B0000E94D5032FEF84E39CE0215080409040BD
:1007C000E1F700C000000C94E91A0F931F93CF9338
:1007D000DF938C0161E00E943B03EC01B8010E94B1
:1007E00003038823F1F1B801CE010E948618882303
:1007F000C1F1B801CE010E949A16882391F1B80187
:10080000CE010E94E217882361F1F80182818823DA
:1008100009F1CB358DE5D807C1F050F4C115FCE5E1
:10082000DF0781F0CF3DDC45A9F40E94700F19C0AD
:10083000CC35EDE5DE0761F0CD35DD4559F40E949C
:10084000AE0E08C00E94D6030CC00E94B70E02C0B4
:100850000E94BA0EC801DF91CF911F910F910C94A5
:10086000010380E0DF91CF911F910F9108950E94C5
:100870001D1A0C9450040E9453040C94231A0895DA
:100880000C943F0481E008950C9442040895CF93A2
:10089000C82F0E9440048C2F0E944404CF910895D9
:1008A00080E00C9447040E94E2180C9447040E94D4
:1008B000E21890918E01891721F080938E010C949B
:1008C00047040895CF93DF93CDB7DEB72B970FB6CC
:1008D000F894DEBF0FBECDBF4F83588769877A87F4
:1008E0008B8761110E94FA0D9E012F5F3F4F86E0BA
:1008F000F90111928A95E9F785E0FE013796D90151
:1009000001900D928A95E1F789819A814C815D81F0
:10091000452B31F09F3F31F491E08F3F19F403C034
:1009200091E001C090E090FF09C049815A816B813C
:100930007C818D819E810E941B0D05C0C9010E9492
:1009400044038111F2CF2B960FB6F894DEBF0FBE91
:10095000CDBFDF91CF910895FC01808191810E94EC
:10096000760A0895CF93882309F4A4C0C82F82384B
:10097000C1F40E94E21881FD9DC069E380910201EB
:10098000909103010E94D8190E941C0E2FEF81EE56
:1009900094E0215080409040E1F700C0000069E3FE
:1009A00019C0833801F50E94E21880FD83C063E519
:1009B00080910201909103010E94D8190E941C0E9F
:1009C0002FEF81EE94E0215080409040E1F700C08D
:1009D000000063E580910201909103010E94E319F8
:1009E000CF910C941C0E8438C1F40E94E21882FD51
:1009F00061C067E480910201909103010E94D819BF
:100A00000E941C0E2FEF81EE94E021508040904018
:100A1000E1F700C0000067E4DDCF8CEF8C0F813A76
:100A2000D0F46C2F80910201909103010E9458191B
:100A3000882349F06C2F80910201909103010E945C
:100A4000E3190E941C0E6C2F80910201909103010A
:100A50000E94D819C5CF80E28C0F883048F4C77047
:100A600081E001C0880FCA95EAF70E94DD0DB8CF7A
:100A7000EBE5EC0FE33040F4F0E0E95BFE4F808102
:100A800090E0CF910C941619E8E5EC0FE73150F4A3
:100A9000F0E0EE0FFF1FE75EFE4F80819181CF9166
:100AA0000C942C19CD3E30F08C2F0E948914CF91DC
:100AB0000C945B15CF910895882309F464C08238A3
:100AC00079F40E94E21881FF5EC069E3809102011F
:100AD000909103010E94D8190E941C0E69E310C076
:100AE0008338B1F40E94E21880FF4DC063E5809125
:100AF0000201909103010E94D8190E941C0E63E527
:100B000080910201909103010E94E3190C941C0E44
:100B1000843879F40E94E21882FF35C067E480913E
:100B20000201909103010E94D8190E941C0E67E4F3
:100B3000E7CF9CEF980F913A10F4682FE1CF90E245
:100B4000980F983050F4877091E001C0990F8A9502
:100B5000EAF7892F0E94E30DD9CF9BE5980F9330D8
:100B600020F480E090E00C94161998E5980F9731E6
:100B700020F480E090E00C942C198D3E20F00E942F
:100B8000E4140C945B1508951F93CF93DF93182FF3
:100B9000EB010E94B204209741F08FE99FE001979A
:100BA000F1F700C000002197F6CF812FDF91CF91A0
:100BB0001F910C945C05893319F060E070E002C06D
:100BC00060E570E00C94C405882321F00E94DD0DDF
:100BD0000C941C0E0895882321F00E94E30D0C94C0
:100BE0001C0E0895CF92DF92EF92FF920F931F9306
:100BF000CF93DF937C01D62FC72FFC011281058193
:100C000002950F700E94D30D8823B9F01123A9F02B
:100C10008C2F807F803421F080E28D0F883068F047
:100C20008091850282FD09C082E00E947C0E0E94B4
:100C3000D30D91E0D82ED92601C0D12CCC2EC29450
:100C40008FE0C8228C2D90E08C30910508F0CFC148
:100C5000FC01E25AFF4F0C94EF218C2F807FCF7064
:100C6000882311F0C295C07F112399F0CC2309F499
:100C7000AAC180E28D0F883010F0D11104C08C2FF2
:100C80000E94DD0D03C08C2F0E94ED0D0E941C0EF2
:100C90009AC18D2F0E945C05CC2309F4A8C180E283
:100CA0008D0F883038F1DD2329F18C2F0E94F30D50
:100CB00024C08C2F807FCF70803211F0C295C07F0E
:100CC000DD2319F0D130A1F13DC08091850282FF72
:100CD00017C0112349F0CC2329F08C2F0E94DD0D81
:100CE0000E941C0E80E070C180E00E945C05CC2355
:100CF00009F47DC18C2F0E94E30D0E941C0E77C168
:100D0000112371F0002341F0013031F40E94FD0DF8
:100D10008C2B0E94050E6BC10E94FD0D8C2B1DC0FB
:100D2000002319F0013009F462C10E94120E25C09F
:100D3000112321F0063008F05AC10EC0053008F02A
:100D400056C11BC0112361F0002331F0F7018581EA
:100D500080FF39C18F7085838C2F0E94E40547C1C5
:100D6000002359F0D93309F03FC1FFEF07EE13E03C
:100D7000F15000401040E1F735C18C2F0E94EB0587
:100D800036C18C2F86958695837019F0813061F07D
:100D90002EC1112321F08D2F9C2F937002C080E073
:100DA00090E00E9416192BC1112321F08D2F9C2F4A
:100DB000937002C080E090E00E942C1920C18D2F1A
:100DC000112319F00E94891402C00E94E4140E94A9
:100DD0005B1515C18C2F837009F047C011110BC131
:100DE0002D2F229526952770220F220F6D2F6F70C1
:100DF000862F90E0A0E0B0E0022E04C0880F991F7B
:100E0000AA1FBB1F0A94D2F7D4FF10C04FE050E0D6
:100E100060E070E004C0440F551F661F771F2A95DD
:100E2000D2F7409550956095709503C040E050E032
:100E3000BA01C695C695C3708A019B01082B192B70
:100E40002A2B3B2BC901B801C23049F058F4C130FC
:100E500019F00E94F308CFC00E94E108CCC00E94A4
:100E60000509C9C00E94DF08C6C0112319F08C2FE4
:100E7000817001C08695882309F4BDC02D2F22956D
:100E800026952770220F220F6D2F6F70862F90E00E
:100E9000A0E0B0E0022E04C0880F991FAA1FBB1F5C
:100EA0000A94D2F7D4FF10C04FE050E060E070E049
:100EB00004C0440F551F661F771F2A95D2F740952F
:100EC00050956095709503C040E050E0BA01C6951A
:100ED000C695C3708A019B01082B192B2A2B3B2B2B
:100EE000C901B801C23049F058F4C13019F00E946C
:100EF000B80981C00E94A6097EC00E94CA097BC0B1
:100F00000E94190978C0CF70112339F08C2F0E94EC
:100F10003F098D2F0E94E4056EC08D2F0E94EB05C6
:100F20008C2F0E94600967C0D23F21F128F4D03F86
:100F300041F0D13FC1F043C0D33F19F1D43F79F024
:100F40003EC0112341F0053008F051C08C2F8F7145
:100F50000E9485094CC0063008F049C0F7CF809147
:100F6000850282FF18C0112339F08C2F8F710E94E7
:100F70003F093DC01123C9F38C2F8F710E94600976
:100F800036C0112329F08C2F8F710E942A092FC09F
:100F90000E9425092CC0112349F0CF718C2F0E948B
:100FA0003F0963E08C2F0E94610E21C081E00E9406
:100FB0007C0E0230E0F082E00E947C0E18C011230B
:100FC00031F0002391F28D2F0E94B20410C0002353
:100FD00099F2D93349F41FEF27EE33E01150204046
:100FE0003040E1F700C000008D2F0E945C0588EFC3
:100FF0008C0D843020F40E94E2180E944704DD200A
:10100000C9F00E94CF0D80FD15C0F70112820E9429
:10101000C90D0E943F09C7010E943B080E94C90DEB
:10102000DF91CF911F910F91FF90EF90DF90CF90C4
:101030000C946009DF91CF911F910F91FF90EF9079
:10104000DF90CF9008950F931F93CF93DF93EC0120
:10105000688179818A810E94810A8C010E94DC0961
:101060000E94CD08B801CE010E94F205DF91CF9118
:101070001F910F910895CF93DF93EC01988189819F
:101080002B813C81232B31F08F3F31F481E09F3F56
:1010900019F403C081E001C080E080FD1DC0CE01D5
:1010A0000E94E503811110C00E94D30D8823A1F096
:1010B0008A81882389F08091850282FD0DC082E0BB
:1010C000DF91CF910C947C0ECE010E942308CE01BB
:1010D000DF91CF910C944603DF91CF91089580E08A
:1010E00090E00E94161980E090E00E942C190E9466
:1010F000FA0D0E941C0E0E948C160C945B158091B8
:101100000201909103010E94EE190C946F080E9455
:10111000EA0D0C947F0892959F70963079F010F448
:10112000925001C09A50923068F4803F69F018F4F0
:10113000883E40F409C0843F29F406C0883E20F070
:10114000813F11F080E0089581E00895FC018081E5
:1011500091810E94760A0E948B080895CF93DF93B5
:1011600000D000D01F92CDB7DEB70F900F900F9038
:101170000F900F90DF91CF910895CF93DF9300D020
:1011800000D000D0CDB7DEB726960FB6F894DEBFFC
:101190000FBECDBFDF91CF910895089508950C94AF
:1011A000CE080C94CF080E94D1086093B2017093CE
:1011B000B3018093B4019093B5010C946F080C9423
:1011C000D3080F931F930091B2011091B3012091A6
:1011D000B4013091B501602B712B822B932B1F91A1
:1011E0000F910C94D3080F931F930091B2011091AB
:1011F000B3012091B4013091B501602371238223A2
:1012000093231F910F910C94D3080F931F93009178
:10121000B2011091B3012091B4013091B501602762
:101220007127822793271F910F910C94D3080C9458
:10123000CE080E9417096093AE017093AF018093AE
:10124000B0019093B1010C946F0860E070E0CB01A5
:101250000C9419090F931F9341E050E060E070E097
:101260008A019B0104C0000F111F221F331F8A95A2
:10127000D2F7C901B8011F910F910C9419090F936E
:101280001F9341E050E060E070E004C0440F551F40
:10129000661F771F8A95D2F78091AE019091AF01BA
:1012A000A091B001B091B1018A019B01082B192BCB
:1012B0002A2B3B2BC901B8011F910F910C941909DE
:1012C0000F931F9341E050E060E070E004C0440FD2
:1012D000551F661F771F8A95D2F7409550956095E8
:1012E00070958091AE019091AF01A091B001B09145
:1012F000B1018A019B01082319232A233B23C90139
:10130000B8011F910F910C9419090F931F9341E09D
:1013100050E060E070E004C0440F551F661F771F67
:101320008A95D2F78091AE019091AF01A091B00162
:10133000B091B1018A019B01082719272A273B2771
:10134000C901B8011F910F910C9419090F931F93B4
:101350000091AE011091AF012091B0013091B10127
:10136000602B712B822B932B1F910F910C941909D9
:101370000F931F930091AE011091AF012091B00126
:101380003091B10160237123822393231F910F9128
:101390000C9419090F931F930091AE011091AF01A6
:1013A0002091B0013091B1016027712782279327E6
:1013B0001F910F910C94190908952CE0929F800DB4
:1013C0001124E82FE695E695E695877051E001C077
:1013D000550F8A95EAF785E0E89FF0011124E05760
:1013E000FE4F20E030E070E04081CB01022E02C0D1
:1013F000969587950A94E2F78170819584278523D5
:10140000842781932F5F3F4F2530310569F7089579
:101410002CE0929F800D1124682F66956695669545
:10142000982F977085E0689FB001112440E050E04C
:1014300080E0FB01E40FF51FE057FE4F208130E014
:10144000092E02C0369527950A94E2F721703327BA
:10145000042E01C0220F0A94EAF7822B4F5F5F4FE0
:101460004530510531F70895BF92CF92DF92EF9248
:10147000FF920F931F93CF93DF938C01C090AE0127
:10148000D090AF01E090B001F090B1018091B20135
:101490009091B301A091B401B091B501C82AD92AA5
:1014A000EA2AFB2ACFE1D0E0D701C6010C2E04C006
:1014B000B695A795979587950A94D2F780FD04C0B5
:1014C000219790F7B12C07C0BC2EB8018C2F0E9439
:1014D00082110197A9F38B2DDF91CF911F910F916D
:1014E000FF90EF90DF90CF90BF900895CF93DF9360
:1014F000EC010E94340ABE010E948211DF91CF915B
:1015000008951F93CF93DF93EB0190918F0199235F
:1015100021F0CB010E94760A13C0882349F0CB0149
:101520000E94340A182F682FCE010E94DD0904C0E2
:10153000CB010E94080A182FBE01812F0E94821140
:10154000DF91CF911F9108951F93CF93DF93C091A7
:10155000B60116E08091B701C81799F0D0E01C9F42
:10156000F0011D9FF00D1124E854FE4F4081518180
:1015700062817381848195810E94BD082196C77024
:10158000E9CFDF91CF911F9108954091E8015091EB
:10159000E9016091EA017091EB018091EC01909179
:1015A000ED010C94BD08EF92FF920F931F93CF9320
:1015B000DF938091ED0182958F7009F065C0809175
:1015C000EA01882309F460C08091B601F090B70168
:1015D0001091E8010091E9016091EB017091EC013B
:1015E00091E01F3F09F090E0C0910001D09101010E
:1015F000292F96E0E92E8F1509F446C06115710573
:1016000021F00F3F21F030E003C031E001C0322F64
:1016100090E030FD36C0E89EF001E99EF00D112407
:10162000DF01A854BE4F11963C911197301329C089
:101630003C91311326C012963C911297311121C072
:1016400013964D915C911497461B570B4C175D07F1
:10165000C0F48091ED018F7080618093ED01E354BF
:10166000FE4F80818F708061808388EE91E00E94C0
:101670003B08DF91CF911F910F91FF90EF900C9459
:10168000A40A01968770B7CFDF91CF911F910F9178
:10169000FF90EF9008959F92AF92BF92CF92DF920A
:1016A000EF92FF920F931F93CF93DF93CDB7DEB7E7
:1016B00061970FB6F894DEBF0FBECDBF8C0185E0F9
:1016C000F801DE011D9601900D928A95E1F7D8018F
:1016D0001296EC909091E801E091E9012091EB01E4
:1016E0003091EC012115310531F0EF3F31F481E00B
:1016F0009F3F19F403C081E001C080E0B82FB170B2
:101700009B2E80FD47C1D8014C9111965C91119799
:101710001396AD90BC90149788EEC82E81E0D82E19
:10172000F090EA01B501621B730B2091000130912A
:101730000101FF2009F4D9C08091ED016217730700
:1017400008F095C0282F207F09F052C05E1313C007
:10175000491311C0FE2CE1100EC08F708061809380
:10176000ED010E94C50AC6010E943B088091ED016F
:10177000F80185834DC1AB2831F05F3F31F481E042
:101780004F3F19F403C081E001C080E080FD03C039
:1017900081E08E2502C080E090E0F82FF170FF2EEE
:1017A00080FF1CC08091B6012091B70136E08217FE
:1017B00009F40BC190E0389FF001399FF00D11241E
:1017C000E854FE4F6181561306C06081461303C082
:1017D0006281E61203C001968770E9CFFE2CEE20ED
:1017E00009F416C18091ED0181608093ED0154C030
:1017F0005E1306C0491304C0E11002C0F80199C08D
:10180000C8010E94A608882361F1EE2051F12091C1
:10181000ED01822F82958F7090E0029774F0809195
:10182000E8019091E90198878F831986BB86AA8683
:101830002C87CE0107960E943B0886E0F801A8EEAF
:10184000B1E001900D928A95E1F70E94D30A0E94BF
:10185000C50A0AC05E1711F1C8010E94A6088111CD
:101860002CC0C8010E943B08FF24F394D1C0282F4C
:10187000207F81F77A2DB98AA88A6E2D89890E94E6
:10188000AE0888EE91E00E943B0886E0D6011D92EA
:101890008A95E9F70E94C50AF12CBAC04913DCCF3A
:1018A000E110DACFF8018583C8010E943B0886E089
:1018B000D6011D928A95E9F7ABC0EE2091F22091F6
:1018C000ED01822F82958F7090E002970CF4B5CFD6
:1018D0008091E8019091E9019A8389831B82BD82FE
:1018E000AC822E83CE010196A6CF6217730708F053
:1018F00044C0FE2CEE2009F4B4CF5E1330C049136F
:101900002EC02091ED0120FD21C0822F82958F7085
:10191000482F50E041155105C9F0F80125834F309B
:10192000510541F08F5F982F9295907F822F8F7095
:10193000892B8583C8010E943B0886E0F801A8EE48
:10194000B1E001900D928A95E1F73CC086E0F80184
:10195000A8EEB1E001900D928A95E1F759C0C80157
:101960000E94A608811169CF8091ED01816080936A
:10197000ED01C8010E943B084BC07A2DB98AA88AA4
:101980006E2D89890E94AE0886E0D6011D928A9547
:10199000E9F718C0EE2009F464CFC8010E94A60838
:1019A000F82E882309F45DCF86E0F801A8EEB1E0B7
:1019B00001900D928A95E1F788EE91E00E94AC04C7
:1019C0000E94D30A0E94C50A23C04D875E878D8579
:1019D0009E850E94760A292F22952F70223028F4A6
:1019E0009F7039F0811105C00BC0243028F49F701E
:1019F00049F4805E883020F0C8010E943B089F2C8B
:101A0000F92C06C0D80115969C91907F91F7F8CFDC
:101A10008F2D61960FB6F894DEBF0FBECDBFDF915C
:101A2000CF911F910F91FF90EF90DF90CF90BF90DB
:101A3000AF909F9008951F93CF93DF93CDB7DEB7FC
:101A40002C970FB6F894DEBF0FBECDBF4F835887DB
:101A500069877A878B879C87CE0107960E944B0BFC
:101A60008823D1F09F8188852A853B85232B31F0FF
:101A70008F3F31F481E09F3F19F403C081E001C042
:101A800080E080FD47C04F81588569857A858B85C8
:101A90009C850E94BD083EC086E0FE013796DE01AF
:101AA000119601900D928A95E1F7FF81E8856A858C
:101AB0007B856115710531F0EF3F31F481E0FF3F27
:101AC00019F403C081E001C080E080FD23C02091B3
:101AD000B70130E0C9010196877099274091B6019E
:101AE00050E084179507F1F1F983EA837D836C83D5
:101AF00096E0929FD001939FB00D1124A854BE4F41
:101B0000FE01319601900D929A95E1F78093B7010D
:101B10000E94A40A16E08091B6019091B70189173E
:101B200071F1189FC001112488549E4F0E944B0BE5
:101B3000882329F1E091B6011E9FF0011124E85499
:101B4000FE4F4081518162817381848195810E9421
:101B5000BD088091B60190E0019687709927809327
:101B6000B601D9CF0E9487081092B7011092B60132
:101B7000E8EEF1E086E0DF011D928A95E9F72C9608
:101B80000FB6F894DEBF0FBECDBFDF91CF911F918E
:101B9000089580910E02859585958595089580918B
:101BA0000E028770089590910E02977081E009F4FB
:101BB00080E0089580913102089590913102892B3F
:101BC000809331020895809590913102892380930A
:101BD0003102089510923102089590913002892BBC
:101BE00080933002089580959091300289238093EC
:101BF0003002089510923002089580910F020895E6
:101C000008950C94000E0C94010E9091850292FDA3
:101C100008C090910F02981721F080930F020C9446
:101C2000030E089580910F02882329F010920F026D
:101C300080E00C94030E0895CF93DF93E0910201AE
:101C4000F0910301809131028083E0910201F091D3
:101C50000301908180913002892B808380910F0253
:101C6000882381F0E0910201F09103019081892B9A
:101C7000808380910201909103010E944219811199
:101C80000E94120EC0910201D091030140E250E087
:101C90006EEE71E0CE010E940922892B69F080E28C
:101CA000FE01AEEEB1E001900D928A95E1F7CE0112
:101CB000DF91CF910C94EE18DF91CF9108950C94A1
:101CC000000E9091850292FD10C098E0899F9001CE
:101CD0001124262B20930E020E943F0980910E02B0
:101CE0008595859585950C945F0E0C943F0910920F
:101CF0000E0280E00C945F0E20910E0280958223EC
:101D000080930E02982F977099F430E0482F082E98
:101D1000000C550B2417350759F09091850292FD60
:101D200007C08595859585950E9460090C94770E6E
:101D300008959091850292FB222720F9281769F0D7
:101D400080FB92F9909385028091840290918502A4
:101D50000E94EC0E82E00C947C0E08958091850226
:101D600082FB882780F991E089270C94990E81E005
:101D70000C94990E80E00C94990E6FEF7FEF80E049
:101D800090E00C94422280E090E00E941E2221E02C
:101D9000893E9E4F09F020E0822F089582E090E076
:101DA0000C94162283E090E00C941622682F83E0B6
:101DB00090E00C942422CF9384E090E00E941622BD
:101DC000C82F82E290E00E9416222C2F30E0A90159
:101DD000582BCA01CF910895CF93C92F682F84E063
:101DE00090E00E9424226C2F82E290E0CF910C942C
:101DF0002422AB01BC018FE090E00C943622AB01B1
:101E0000BC0183E190E00C94362260E070E0CB01ED
:101E10000C94FF0E60E070E0CB010E94F90E0C9470
:101E2000050F69EE7EEF80E090E00E94422260E0C4
:101E300082E090E00E94242260E083E090E00E9433
:101E400024221092B2011092B3011092B4011092A8
:101E5000B50160E084E090E00E94242260E082E22C
:101E600090E00E94242260E085E090E00E9424221D
:101E700060E086E090E00E9424226FEF87E090E02F
:101E80000E94242240E050E0BA0188E090E00E94E5
:101E9000362260E08DE090E00E94242240E050E095
:101EA000BA0188E190E00E94362260E087E190E08C
:101EB0000E94242240E050E0BA018CE190E00E94B0
:101EC000362260E070E080E290E00E94422240E032
:101ED00050E0BA0188E190E00E9436220C940A0F8B
:101EE0000C94110F682F8EE090E00C9424220E9435
:101EF000A81A60933E0270933F0280934002909331
:101F0000410260933A0270933B0280933C029093AB
:101F10003D02089585B7806885BF85B7806885BF15
:101F2000089581E008950C94910F08950C94950FF5
:101F30000C94950F0C94980F0C94950F0C949C0F87
:101F40000C94950F0E948A0F8EE592E10E94D8189A
:101F50000E94A00F0C949E0F0E94960F0C94950F58
:101F60000E9478120C9446040E94931A0E945D13FA
:101F70000E94B00F0C949A0F5F926F927F928F9293
:101F80009F92AF92BF92CF92DF92EF92FF920F9308
:101F90001F93CF93DF93CDB7DEB72A970FB6F89490
:101FA000DEBF0FBECDBF0E947213C82E81110E94EA
:101FB000770F32E3832E32E0932E00E010E0502EB4
:101FC000802F0E949C125C01F401619071904F017E
:101FD0006826792661147104B1F40F5F1F4F043035
:101FE000110569F78FEF89838A831B820E949C1AEF
:101FF0008160782F9D838C8349815A816B818D818B
:102000000E9462043AC08091420281FD0E94A512A2
:10201000D12CEE24E394F12CC3018E219F21892B36
:1020200029F10E94930F8823A9F0DE825F82AE20FF
:10203000BF2081E0AB2809F480E088870E949C1AC9
:102040008160782F9A8789874E815F8168858A852C
:102050000E946204000F111FF801EE5CFD4F8081A9
:102060009181E826F926F182E08207C0D394EE0C34
:10207000FF1CFCE0DF12D0CFB0CF81E0C11001C067
:1020800080E02A960FB6F894DEBF0FBECDBFDF9179
:10209000CF911F910F91FF90EF90DF90CF90BF9065
:1020A000AF909F908F907F906F905F9008950E9467
:1020B000BC0F0E9479150C945704CF93DF930E94B4
:1020C0008711EC01811521E5920708F045C08115C3
:1020D00030E5930708F094C0883E910528F5803ECE
:1020E000910508F0F8C0883A910570F4853A910599
:1020F00008F07CC08130910509F475C008F4E8C08F
:10210000049708F0E8C0E4C08F3B910508F0E0C0F8
:10211000C85AD0E0CC0FDD1FC65BDE4F0990D881D6
:10212000C02DCE019464D8C0811540E2940758F4C4
:10213000811551E0950708F0CEC08D3E910508F459
:10214000C7C09065C9C0C11580E4D80708F4C0C0F5
:10215000DF70CE01906AC0C0811525E59207A8F412
:10216000811534E5930708F095C0811543E5940780
:1021700008F07BC0811552E5950708F061C0D82FA3
:10218000CC27CE01816F906AA7C0C11589E5D80719
:10219000A0F4C11528E5D20708F082C0C11536E5C4
:1021A000D30708F095C08C2F0E941B128F7190E00E
:1021B000D82FCC27CE0190628FC0C1154AE5D40735
:1021C00008F474C0CE0190568115904208F080C08A
:1021D0008D2F8F710E941B12DD27D0628F71AE018F
:1021E000582BCA0179C081E090E076C0C55AD0E092
:1021F000C858DE4F8881C82FD0E0CE0190646CC0F3
:1022000074E0969587957A95E1F7282F23703C2FF7
:10221000337081E090E002C0880F991F3A95E2F791
:102220009C68AC01522B9A019C2F9F7096959695B5
:1022300050E2959FE0011124C9018C2B9D2B4CC0CD
:102240008370992721E030E002C0220F331F8A9566
:10225000E2F79C2F9695969580E2989FE0011124D5
:10226000C22BD32BCE019C6837C08370992721E005
:1022700030E002C0220F331F8A95E2F79C2F96951B
:10228000969540E2949FE0011124C22BD32BCE01FE
:102290009A6822C0D82FCC27CE01846F906A1CC0C8
:1022A000DC2FCC27CE01806F906A16C08C2F8F70E8
:1022B0000E941B1294E0D695C7959A95E1F7CF70CE
:1022C000D0E0DC2FCC27D0699E01282BC90104C0A7
:1022D00080E090E001C0CE01DF91CF91089520E32E
:1022E000829FC0011124FC012CE0729FE00DF11DC2
:1022F0001124E60FF11DEE0FFF1FE851FF4F8591EE
:10230000949108950E946F110E945D100895823883
:10231000910569F1B0F48133910509F46DC048F479
:102320008932910509F463C08A32910509F469C0C4
:1023300008958533910509F455C089339105B9F0A5
:102340000895833E910569F138F4803E9105B1F01E
:10235000823E910509F10895863E9105A9F1873ED7
:102360009105B9F1843E910509F064C023C0209124
:10237000840220FD4FC021FD4DC00895809184024C
:1023800080FD44C08091850280FF44C0809184021A
:1023900084FD42C083EE4DC08091840282FF38C02C
:1023A000F5CF8091840282FD33C08091850280FD4B
:1023B00031C0ECCF8091850281FF32C080918402D0
:1023C00084FD2AC087EE35C08091840283FF26C039
:1023D000F5CF8091840283FD21C08091850281FD2B
:1023E0001FC0ECCF8091840285FD1CC01DC0809170
:1023F000840285FD19C016C08091840286FD16C036
:1024000017C08091840286FD13C010C089E311C0FB
:1024100082EE0FC080EE0DC080E00BC086EE09C0DA
:1024200084EE07C089E205C085E303C08AE201C0EB
:1024300081E390E008959091840292FF0DC0282FCF
:102440002871283019F4877F846006C0282F2471F2
:10245000243011F48B7F886093FF0DC0282F2871E2
:10246000283119F4877E846106C0282F2471243115
:1024700011F48B7E88612091850220FF0DC0382FDA
:102480003871383019F4877F816006C0382F317178
:10249000313011F48E7F886021FF0DC0282F287104
:1024A000283119F4877E816106C0282F21712131DE
:1024B00011F48E7E886194FD877E089580E00895F2
:1024C0000C94BD0E0E9472138FE39CE90197F1F703
:1024D00000C000000E94721380E00E949C1280FFE6
:1024E00004C00E9460120C94E91A08950C946212C0
:1024F0000E94C30E811102C00E94700F0E94CE0E76
:10250000809342020E94DB0E9093850280938402A6
:102510000E9476120E94D20E682F70E080E090E058
:102520000E94DF086091AE017091AF018091B0010F
:102530009091B1010C941709E82FF0E0EE0FFF1F06
:10254000E257FD4F808191810895089580EA8A9530
:10255000F1F7089500C008950C94A61208950C9404
:10256000AE120C94AF120C94AE120C94B312F894F9
:10257000E82FE295EF70F0E031A1282F2F7081E075
:1025800090E001C0880F2A95EAF7982F9095932341
:1025900091A392A1892B82A3789408950F931F93FE
:1025A000CF93DF93C7E8D1E089918F3F11F00E946C
:1025B000B71281E0CB38D807B9F7CBE7D1E007E80D
:1025C00011E089918F3F11F00E94B7120C171D077F
:1025D000C1F7DF91CF911F910F910895BF92CF92D4
:1025E000DF92EF92FF920F931F93CF93DF938C01B3
:1025F000C62FD0E0CE0189579E4F6C01FC0190811F
:102600009F3F09F450C0B62EF894E92FE295EF7081
:10261000F0E081A19F7021E030E001C0220F9A9587
:10262000EAF7822B81A382A12095282322A3789404
:102630000E94AA12EBE7F1E047E851E021E030E028
:10264000E12CF12C61916F3F89F0A62FA295AF701C
:10265000B0E090968C9190E06F7002C09595879550
:102660006A95E2F780FD02C0C90102C080E090E0F7
:10267000E82AF92A220F331F4E175F0719F7F601D0
:1026800080818F3F11F00E94B71261E0E114F104E4
:1026900009F460E08B2D0E94AC12CC0FDD1FC00F3F
:1026A000D11FF982E882DF91CF911F910F91FF90A6
:1026B000EF90DF90CF90BF9008950E94CE1288E0F7
:1026C000EEE8F2E0DF01982F1D929A95E9F7E6E82F
:1026D000F2E0DF011D928A95E9F784E00E94BD13C4
:1026E0000C94D103FF920F931F93CF93DF93CDB739
:1026F000DEB728970FB6F894DEBF0FBECDBF8E01B0
:102700000F5F1F4F88E0F80111928A95E9F7F12CCD
:102710006F2DC8010E94EE12F394F4E0FF12F8CF7F
:1027200048E050E0B80186E892E00E940922FF24C8
:10273000F394009709F4F12C892B41F088E0F8011B
:10274000A6E8B2E001900D928A95E1F72F2D44E0C2
:102750006EE872E086E892E00E94BE130E94D30306
:102760008F2D28960FB6F894DEBF0FBECDBFDF9138
:10277000CF911F910F91FF9008950895FF920F93AD
:102780001F93CF93DF93F82E092F162FD72FC42F27
:10279000222349F081E0809345020E949C1A909385
:1027A000440280934302809145028823D9F08091AE
:1027B0004302909144020E94B41A059798F0EF2DBD
:1027C000F02FA12FBD2F80E090E04C2F50E0841718
:1027D000950734F4219131912D933D930196F7CFD4
:1027E00010924502DF91CF911F910F91FF900895B4
:1027F0000E94A11C0E94B40F0C94AD1C0E94B11C3D
:102800000E9457100C94CB1C0E943A1A0E94881CFC
:102810000E94A20F0E94F8130E94FE130E94AC0FA8
:10282000FBCF80914C0280FF06C06091090170E0EF
:10283000660F771F26C081FF04C06091090184E004
:1028400005C082FF07C06091090188E0689FB00160
:10285000112417C090914B029923D1F06091080187
:10286000961788F72091090188E0289F900111248C
:10287000929FA001939F500D112470E0CA010E9405
:10288000DB216038710540F46115710519F406C04B
:1028900068E070E0862F08958FE7089581E008953D
:1028A00080914C0280FF08C06091050170E0759531
:1028B00067957595679521C081FF06C060910501F8
:1028C00070E07595679519C082FF04C0609105019D
:1028D00070E010C090914A02992399F06091040130
:1028E0009617A0F780910501899FC001112470E01F
:1028F0000E94DB216038710540F46115710519F4FF
:1029000006C061E070E0862F08958FE7089581E0AA
:1029100008958D3E21F40E941114819504C08E3ECD
:1029200029F40E9411148093500208958F3E21F4DF
:102930000E941114819504C0803F29F40E94111453
:1029400080934F020895893F19F40E94501405C0E6
:102950008A3F31F40E94501481958093510208956A
:102960008B3F21F40E945014819504C08C3F29F4C0
:102970000E9450148093520208959FE0980F98305F
:1029800078F421E030E0A90102C0440F551F9A9568
:10299000E2F7CA0190914E02892B80934E0208956E
:1029A0008D3F21F480914C0281600BC08E3F21F459
:1029B00080914C02826005C08F3F29F480914C02C7
:1029C000846080934C0208958D3E39F490915002BA
:1029D00097FF35C01092500259C08E3E29F4909155
:1029E00050021916BCF32BC090914F028F3E29F470
:1029F00097FF25C010924F0249C0803F19F4191665
:102A0000CCF31DC090915102893F29F41916BCF4F2
:102A1000109251023BC08A3F19F497FF10C0F8CFC3
:102A20008B3F39F49091520297FF09C010925202E5
:102A30002DC08C3F21F4909152021916BCF39FE0F7
:102A4000980F983080F421E030E0A90102C0440FD3
:102A5000551F9A95E2F7CA01809590914E028923FD
:102A600080934E0213C08D3F21F480914C028E7FE3
:102A70000BC08E3F21F480914C028D7F05C08F3FAB
:102A800029F480914C028B7F80934C0280914F02FD
:102A9000811106C080915002811102C010924B0238
:102AA00080915102811106C080915202811102C0B1
:102AB00010924A0208950E949C1A20914F022111FF
:102AC00004C020915002222321F090934902809368
:102AD000480220915102211104C020915202222368
:102AE00021F090934702809346028DE492E00C948B
:102AF0000819EF92FF920F931F93CF93DF9300D0AB
:102B000000D000D0CDB7DEB786E0EDE4F2E0DE0124
:102B1000119601900D928A95E1F7E0904F02F090A6
:102B20005002009151021091520210924F021092E5
:102B300050021092510210925202E11003C0FF2085
:102B400009F45DC080914802909149020E94B41A34
:102B5000AC0190914B02992339F020910A0130E0A9
:102B60002417350758F04BC020910B018AE0289FAD
:102B7000900111242417350718F041C09F3F19F028
:102B80009F5F90934B02EE2061F00E9411141E147F
:102B900014F09FEF01C091E0989F902D1124909325
:102BA0004F02FF2061F00E9411141F1414F09FEFD8
:102BB00001C091E0989F902D112490935002309184
:102BC0004F023323E1F0209150022223C1F045EB64
:102BD0003403C0011124992319F090934F0203C0CC
:102BE00081E080934F0235EB2303C0011124992328
:102BF00019F09093500203C081E0809350020111BC
:102C000003C0112309F45DC08091460290914702F0
:102C10000E94B41AAC0190914A02992339F0209194
:102C2000060130E02417350758F04BC0209107010A
:102C30008AE0289F900111242417350718F041C01D
:102C40009F3F19F09F5F90934A02002361F00E941A
:102C50005014101614F09FEF01C091E0989F902D32
:102C6000112490935102112361F00E945014111607
:102C700014F09FEF01C091E0989F902D1124909344
:102C80005202309151023323E1F02091520222236B
:102C9000C1F045EB3403C0011124992319F090933E
:102CA000510203C081E08093510235EB2303C00140
:102CB0001124992319F09093520203C081E080936C
:102CC000520280914F0281110BC0809150028111FC
:102CD00007C080915102811103C08091520281117D
:102CE0000E945B15EB82FC820D831E8386E0FE0151
:102CF0003196ADE4B2E001900D928A95E1F7269607
:102D00000FB6F894DEBF0FBECDBFDF91CF911F91FC
:102D10000F91FF90EF900895EDE4F2E086E0DF017F
:102D20001D928A95E9F710924B0210924A02109276
:102D30004C020895CF93DF93EC01FB01828188233D
:102D400009F43CC1C430FDE5DF0760F4CB3F9CE5EE
:102D5000D90788F49E0122503C452431310508F002
:102D60002EC109C0C236EDE5DE0729F0C63AFDE501
:102D7000DF0709F024C10E94DB0E90938502809347
:102D80008402C1318CE5D80709F4C6C008F042C0FE
:102D9000C930ECE5DE0709F49BC000F5C5308CE5D1
:102DA000D80709F485C078F4C330ECE5DE0709F4F0
:102DB00078C008F07AC0C230DC4509F0F5C08091D7
:102DC00084028160EFC0C7309CE5D90709F478C060
:102DD00008F07AC0809184028061E4C0CD30FCE5C7
:102DE000DF0709F487C058F4CB309CE5D90709F414
:102DF00079C008F07BC08091840288606FC0CF30BA
:102E0000FCE5DF0709F480C008F082C080918402ED
:102E1000877FC8C0CE3F9CE5D90709F471C000F593
:102E2000C531FCE5DF0709F485C068F4C3319CE5D2
:102E3000D90709F475C008F095C00E9487088091F1
:102E400084028F77AFC0CC3FFCE5DF07A9F108F023
:102E500054C0CB3FDC4509F0A7C08091850240C03B
:102E6000C230EDE5DE0709F489C058F4C1158DE5DF
:102E7000D80709F45AC008F069C0809185028260C1
:102E80002FC0C236EDE5DE0709F47CC0C63AFDE589
:102E9000DF0709F481C0C330DD4509F085C080E05B
:102EA0006EC08091840282607DC08091840216C0D1
:102EB00080918402886076C08091850282604FC0D4
:102EC0008091840280626EC08091840280646AC0B6
:102ED0000E94870880918402806864C0846062C018
:102EE00081603DC0809184028E7F5CC080918402AD
:102EF0008D7F58C08091840216C08091850218C0D1
:102F0000809185028D7F2BC0809184028F7E4AC084
:102F1000809184028F7D46C0809184028F7B42C065
:102F200080918402877F8B7F3DC0809185028D7F59
:102F30008E7F15C08091840282FB222720F991E0C8
:102F4000922790FB82F990FB83F92CC08091850237
:102F5000982F909591708E7F892B90FB81F98093AB
:102F6000850222C00E9487088091840287FB222765
:102F700020F991E0922790FB87F914C081E00E942C
:102F8000720F12C08091840284FB222720F991E005
:102F9000922790FB84F906C080918402982F909527
:102FA00090FB80F980938402809184029091850245
:102FB0000E94EC0E0E94870880E001C081E0DF9152
:102FC000CF910895CF93DF9386319C4541F5EB0176
:102FD0000E94DA0D982F8A8120910201309103011D
:102FE000882379F09A7A81E009F480E08093530293
:102FF000911102C069E201C065E3C9010E94D819BC
:103000000AC080915302811102C069E201C065E3E8
:10301000C9010E94E3190E941C0E80E001C081E0FA
:10302000DF91CF9108950F931F93CF93DF93C42F18
:10303000D22FFC0182818823C9F0409356020E945E
:103040009C1A909355028093540280E28C0F883032
:1030500008F057C0C77081E001C0880FCA95EAF731
:10306000DF91CF911F910F910C94E405809156024E
:10307000481330C080915402909155020E94B41AB6
:10308000883C910538F510E21D0FCD17B9F080E2AC
:103090008C0F883040F4C77081E001C0880FCA955A
:1030A000EAF70E94EB05183028F581E09D2F977014
:1030B00001C0880F9A95EAF70E94E405802F0E94CC
:1030C000DB051830F0F4D77081E001C0880FDA9585
:1030D000EAF70AC080E28C0F883098F4C77081E06C
:1030E00001C0880FCA95EAF7DF91CF911F910F9128
:1030F0000C94EB05802FDF91CF911F910F910C94D1
:10310000DB05DF91CF911F910F9108950F939C01E3
:10311000CB01243F4CE5340731F188F4293DFCE52F
:103120003F07D9F02A3D4CE5340779F1283D3C456D
:10313000A9F506E221EE41EE68ED7CE52BC0263FC5
:10314000FCE53F07E1F0A8F0273F3C4539F507E2F1
:1031500025EE46EE67EF7CE51DC007E225EE45EE65
:1031600069ED7CE517C006E221EE40EE64EF7CE5F8
:1031700011C007E225EE44EE65EF7CE50BC006E2E8
:1031800021EE42EE66EF7CE505C008E221E045EE67
:103190006AED7CE50E94131880E008C0FC01828182
:1031A000882319F01092560201C081E00F91089512
:1031B00090938D0180938C01089590935C0280938D
:1031C0005B020895E0915B02F0915C02309721F080
:1031D0000190F081E02D099480E00895E0915B0278
:1031E000F0915C02309799F020911801222359F058
:1031F0002091840227FF07C0DC012C9111962C93AB
:10320000119726E02C930280F381E02D0994089514
:10321000E0915B02F0915C02309739F022E0DC0132
:103220002C930480F581E02D099408952091590292
:1032300030915A022817390771F090935A028093FF
:103240005902E0915B02F0915C02309721F0068018
:10325000F781E02D0994089520915702309158028A
:103260002817390771F09093580280935702E09124
:103270005B02F0915C02309721F00084F185E02D33
:1032800009940895FC01329680911801882331F049
:103290008091840287FF02C09EE101C096E080E039
:1032A000915028F021912223D9F38F5FF9CF08950F
:1032B000662351F1209118012223E9F02091840224
:1032C00027FF19C0462F4695469546954E31E0F4A6
:1032D000677021E030E002C0220F331F6A95E2F7E9
:1032E000FC01E40FF11D828190E02823392381E065
:1032F000232B69F409C0FC013296089621916217CC
:1033000029F0E817F907D1F780E0089581E00895E2
:103310009C01FC0132969FEF80E04191461789F0B5
:103320009F3F19F4411101C0982F8F5F8630A9F794
:103330009F3F39F0F901E90FF11D97FDFA9562837E
:10334000089508959C012A5F3F4FFC014281461376
:1033500001C01282019682179307B9F70895262FAC
:103360002695269526952E3168F4FC01E20FF11D75
:10337000677021E030E001C0220F6A95EAF7828190
:10338000282B22830895262F2695269526952E31C3
:1033900070F4FC01E20FF11D677021E030E001C024
:1033A000220F6A95EAF720958281282322830895C7
:1033B00020911801222329F02091840227FD0C94EA
:1033C000AF190C94881920911801222329F020911B
:1033D000840227FD0C94C3190C94A21920911801A2
:1033E000FC013296222331F08091840287FF02C0D3
:1033F0008EE101C086E0DF011D928A95E9F708950C
:1034000008950C94001A83E080935D020C94011AD5
:10341000811102C081E001C082E080935D020C94C2
:10342000011A0C94081A81E080935D020C94011A31
:103430000C94131A08950C941A1A0C941B1A0C94D9
:103440001A1A0C941A1A0C941A1ACF930E94211A61
:103450000E9472130E941F1AC0E08C2F0E949C12BF
:10346000892B29F4CF5FC430C1F780E001C081E02F
:10347000CF91089508951F920F920FB60F921124C5
:103480008F939F93AF93BF9380915E02811113C07E
:103490008091960290919702A0919802B091990222
:1034A0004196A11DB11D8093960290939702A0931F
:1034B0009802B0939902BF91AF919F918F910F9015
:1034C0000FBE0F901F90189580919E02843031F1AD
:1034D0000E94370410925E0220E488E190E00FB66B
:1034E000F894A895809360000FBE2093600083B786
:1034F000817F846083BF83B7816083BF7894889520
:1035000083B78E7F83BF0FB6F894A8958091600033
:10351000886180936000109260000FBE08950E9441
:1035200087080C943B0482E084BD93E095BD9AEF3C
:1035300097BD80936E0008952FB7F89480919602FE
:1035400090919702A0919802B09199022FBF08958F
:103550002FB7F8946091960270919702809198022B
:10356000909199022FBF08959C014FB7F8948091D4
:10357000960290919702A0919802B09199024FBF44
:10358000821B930B089578941F920F920FB60F929F
:1035900011248F939F93AF93BF9380919602909144
:1035A0009702A0919802B09199020196A11DB11DB8
:1035B0008093960290939702A0939802B0939902F9
:1035C000BF91AF919F918F910F900FBE0F901F9061
:1035D000189587E797E790930108809300089AE091
:1035E00088E10FB6F894A895809360000FBE909381
:1035F0006000FFCF809182020895089522E0209319
:10360000E9002FEF3091E800215035FD06C035ED7F
:103610003A95F1F700002111F5CF2091E80025FF40
:103620000BC040E050E066E070E00E943D1D8091DC
:10363000E8008E778093E8000895CF93DF93209180
:103640001801222339F02091840227FF03C060E291
:1036500022E002C068E021E02093E9002FEF3091E2
:10366000E800215035FD06C035ED3A95F1F7000030
:103670002111F5CF2091E80025FF1DC0EC018091BC
:103680001801811105C040E050E068E070E003C01F
:1036900070E040E050E0CE010E943D1D8091E800C6
:1036A0008E778093E80080E2FE01A2E6B2E001900E
:1036B0000D928A95E1F7DF91CF91089580935F0293
:1036C000709361026093600280919E02843001F5E4
:1036D00082E08093E9008FEF9091E800815095FDA2
:1036E00006C095ED9A95F1F700008111F5CF809114
:1036F000E80085FF0DC040E050E063E070E08FE53A
:1037000092E00E943D1D8091E8008E778093E80052
:103710000895BC0184E00C945E1BBC0183E00C9412
:103720005E1B80919D02811109C00E94CE1E0E94E5
:103730002B1F8091E20084608093E2000895109234
:103740009D0208950C94181A60919A0281E061110B
:1037500001C080E00C94031A90919E0281E09430A5
:1037600009F080E060919A020C94081A42E061EC42
:1037700081E00E94471E42E261EC82E00E94471E07
:1037800090919E0281E0943009F080E060919A026D
:103790000C94111A8091A002833009F461C030F4B6
:1037A000813071F0823009F49AC008958A3009F4AA
:1037B00086C08B3009F46CC0893009F0A8C020C0E5
:1037C00080919F02813A09F0A2C08091E800877F32
:1037D0008093E8008091A3029091A402892B21F4A8
:1037E00060E282E692E003C060E080E090E070E09A
:1037F0000E94881D8091E8008B778093E8000895EF
:1038000080919F02813209F082C08091A302909141
:10381000A402029708F07BC08091E800877F809324
:10382000E8008091E80082FD05C080919E02811130
:10383000F8CF6DC02091F3008091F20090E0922BC0
:10384000029731F48091F100813011F0863021F43B
:103850008091F100809382028091E8008B7753C0C1
:1038600080919F02813A09F052C08091A302909109
:10387000A402892B09F04BC08091E800877F8093D8
:10388000E8008091E80080FFFCCF8091180136C0ED
:1038900080919F028132D9F58091A3029091A40278
:1038A000892BA9F58091E800877F8093E8000E942A
:1038B0007C1E8091A102809318010C94870880914E
:1038C0009F02813221F58091E800877F8093E80094
:1038D0000E947C1E8091A2028093830208958091B1
:1038E0009F02813AA1F48091E800877F8093E800ED
:1038F0008091E80080FFFCCF809183028093F100EB
:103900008091E8008E778093E8000C947C1E0895E7
:1039100084B7877F84BF0FB6F894A8958091600024
:10392000886180936000109260000FBE90E080E894
:103930000FB6F89480936100909361000FBE0C94D1
:10394000131A0E94CE1E0E942B1FE2EEF0E080812F
:103950008460808378940C94C0218CE091E00C9476
:10396000DD1880919E028530A9F480919E028530F9
:1039700079F40E94641A80919C028823B1F30E941A
:10398000251A882391F30E94271D0E948708EDCFF6
:103990000C948F1A089508950C94CE1C292F332768
:1039A00023303105C9F060F42130310581F0223037
:1039B000310509F044C08BE390E02CEA33E043C0CA
:1039C00021323105E1F02232310549F138C082E17E
:1039D00090E027EE33E037C099278130910549F018
:1039E00028F0029761F5E8E8F3E005C0E8EAF3E0C3
:1039F00002C0E8E9F3E0849190E09F0124C06115E2
:103A0000710541F061307105D1F489E090E027ED56
:103A100033E019C089E090E02EEB33E014C061156B
:103A2000710541F06130710551F486EB90E029EFAA
:103A300033E009C080E490E02FEA34E004C080E085
:103A400090E020E030E0FA0131832083089580E1A6
:103A500089BD82E189BD09B400FEFDCF8091D80007
:103A60008F7D8093D8008091E00082608093E00099
:103A70008091E00081FDFCCF0895CF92DF92EF921C
:103A8000FF920F931F93CF93DF93EC018B017A0189
:103A90000E949B1E811133C0E114F10439F0F7013B
:103AA00080819181081B190BC80FD91FC12CD12C03
:103AB0000115110519F18091E80085FD16C080916E
:103AC000E8008E778093E800E114F10449F0F701F3
:103AD00080819181C80ED91ED182C08285E00FC03D
:103AE0000E949B1E882321F30AC089918093F100D4
:103AF00001501109FFEFCF1ADF0ADACF80E0DF9122
:103B0000CF911F910F91FF90EF90DF90CF9008958C
:103B10002091A5023091A6022617370748F06115BB
:103B2000710539F42091E8002E772093E80001C058
:103B3000B901FC0120E06115710579F180919E02C7
:103B40008823F1F18530F1F18091E80083FD3CC0DC
:103B50008091E80082FD2EC08091E80080FFEBCFCD
:103B60002091F3008091F20090E0922B6115710595
:103B700051F08830910538F421912093F100615083
:103B800071090196F3CF21E0089709F020E08091B8
:103B9000E8008E778093E800CECF2111CFCF0AC006
:103BA00080919E02882361F0853061F08091E80069
:103BB00083FD0AC08091E80082FFF2CF80E0089583
:103BC00082E0089583E0089581E008952091A502A0
:103BD0003091A6022617370748F06115710539F4B0
:103BE0002091E8002E772093E80001C0B901FC0184
:103BF00020E06115710591F180919E02882309F4FE
:103C000040C0853009F43FC08091E80083FD3DC08D
:103C10008091E80082FD2FC08091E80080FFE9CF0D
:103C20002091F3008091F20090E0922B61157105D4
:103C300059F08830910540F424912093F100319699
:103C4000615071090196F2CF21E0089709F020E058
:103C50008091E8008E778093E800CBCF2111CCCF04
:103C60000AC080919E02882361F0853061F08091C6
:103C7000E80083FD0AC08091E80082FFF2CF80E077
:103C8000089582E0089583E0089581E00895982FD3
:103C9000973068F59093E900981739F07091EC002F
:103CA0002091ED005091F00003C0242F762F50E0BA
:103CB00021FD02C09F5FECCF3091EB003E7F30933F
:103CC000EB003091ED003D7F3093ED003091EB0043
:103CD00031603093EB007093EC002093ED00509333
:103CE000F0002091EE0027FDE5CF80E008958F7071
:103CF0008093E90081E0089580919F0287FF11C0C1
:103D00008091E80082FD05C080919E028111F8CF6C
:103D100011C08091E8008B770BC080919E028823B0
:103D200049F08091E80080FFF8CF8091E8008E771D
:103D30008093E80008952091E4003091E50095E635
:103D40004091EC00842F817040FF23C08091E800F7
:103D500080FD1DC080919E02882399F0853099F0E6
:103D60008091EB0085FD11C04091E4005091E50089
:103D70002417350729F3915011F09A01E1CF84E01F
:103D8000089582E0089583E0089581E0089580E039
:103D900008954091E80042FFDDCF08950E943C1F46
:103DA0000E94441FE0EEF0E0808181608083E8EDB6
:103DB000F0E080818F77808319BCA7EDB0E08C9113
:103DC0008E7F8C9380818F7E808310929D020895D8
:103DD0000F931F93CF93DF930E943C1F0E94441FB9
:103DE000C8EDD0E088818F77888388818068888358
:103DF00088818F7D888319BC10929E0210929A024E
:103E000010929C0210929B0200EE10E0F80180815B
:103E10008B7F808388818160888342E060E080E0DE
:103E20000E94471EE1EEF0E080818E7F8083E2EE0B
:103E3000F0E0808181608083808188608083F801E8
:103E400080818E7F8083888180618883DF91CF919C
:103E50001F910F910895E8EDF0E080818F7E8083BF
:103E6000E7EDF0E080818160808384E082BF81E0C3
:103E700080939D020C94E81EE8EDF0E080818E7F37
:103E800080831092E20008951092DA001092E1000F
:103E900008951F920F920FB60F9211242F933F9304
:103EA0004F935F936F937F938F939F93AF93BF9342
:103EB000EF93FF938091E10082FF0BC08091E200BD
:103EC00082FF07C08091E1008B7F8093E1000E9418
:103ED000BF218091DA0080FF1FC08091D80080FF51
:103EE0001BC08091DA008E7F8093DA008091D90028
:103EF00080FF0DC080E189BD82E189BD09B400FE6B
:103F0000FDCF81E080939E020E94911B05C019BCE9
:103F100010929E020E949F1B8091E10080FF19C0B9
:103F20008091E20080FF15C08091E2008E7F809337
:103F3000E2008091E20080618093E2008091D800ED
:103F400080628093D80019BC85E080939E020E9415
:103F5000A41B8091E10084FF30C08091E20084FFC7
:103F60002CC080E189BD82E189BD09B400FEFDCF8E
:103F70008091D8008F7D8093D8008091E1008F7E62
:103F80008093E1008091E2008F7E8093E200809137
:103F9000E20081608093E20080919A02882311F010
:103FA00084E007C08091E30087FD02C081E001C08A
:103FB00083E080939E020E94AC1B8091E10083FF0E
:103FC00029C08091E20083FF25C08091E100877FB6
:103FD0008093E10082E080939E0210929A02809189
:103FE000E1008E7F8093E1008091E2008E7F8093DC
:103FF000E2008091E20080618093E20042E060E0B4
:1040000080E00E94471E8091F00088608093F0005D
:104010000E94A21BFF91EF91BF91AF919F918F9151
:104020007F916F915F914F913F912F910F900FBEB4
:104030000F901F9018951F920F920FB60F92112498
:104040002F933F934F935F936F937F938F939F93A0
:10405000AF93BF93CF93DF93EF93FF93C091E900AA
:10406000CF708091EC00D82FD17080FDD0E81092F5
:10407000E9008091F000877F8093F00078940E949F
:104080005F201092E9008091F00088608093F0003A
:10409000CD2BCF70C093E900FF91EF91DF91CF91CD
:1040A000BF91AF919F918F917F916F915F914F9150
:1040B0003F912F910F900FBE0F901F9018951F9357
:1040C000CF93DF93CDB7DEB7AA970FB6F894DEBFD4
:1040D0000FBECDBFEFE9F2E08091F100819322E0C5
:1040E000E73AF207C9F70E94CA1B8091E80083FFF4
:1040F0002EC180919F029091A002492F50E04A303A
:10410000510508F024C1FA01E659FF4F0C94EF2144
:10411000803821F0823809F01AC108C080919B02D2
:1041200090919C02992389F082600FC08091A30234
:104130008F70873008F00BC18093E9008091EB000D
:1041400085FB882780F91092E9009091E800977F1D
:104150009093E8008093F1001092F100D1C0282FD5
:104160002D7F09F0F4C0882319F0823061F0EFC090
:104170008091A102813009F0EAC0933009F080E01B
:1041800080939C022EC08091A10281112AC080914F
:10419000A3028F702FEF280F263008F0D8C080932D
:1041A000E9002091EB0020FF1CC0933021F48091A6
:1041B000EB00806214C09091EB0090619093EB0053
:1041C00021E030E0A90102C0440F551F8A95E2F7B3
:1041D0004093EA001092EA008091EB00886080939F
:1041E000EB001092E9008091E800877F8093E8005F
:1041F0000E947C1EACC08111AAC01091A1021F7741
:104200008091E3008078812B8093E3008091E80027
:10421000877F8093E8000E947C1E8091E80080FFE9
:10422000FCCF8091E30080688093E300111102C00D
:1042300082E001C083E080939E0289C08058823072
:1042400008F085C08091A1029091A2028C3D53E0BC
:10425000950779F583E08A838AE289834FB7F894DA
:10426000DE01139620E03EE051E2E32FF0E05093B0
:104270005700E49120FF03C0E295EF703F5FEF70BD
:104280008E2F90E0EA3010F0C79601C0C0968D9353
:104290009D932F5F243149F74FBF8091E800877FBE
:1042A0008093E8006AE270E0CE0101960E94881DCA
:1042B00016C06091A3027091A402AE014F5F5F4FE0
:1042C0000E94CC1CBC01892B09F441C09091E800EC
:1042D000977F9093E80089819A810E94E61D8091E2
:1042E000E8008B778093E80032C0803881F58091B8
:1042F000E800877F8093E80080919A028093F10024
:104300008091E8008E7772CF811121C08091A10247
:104310009091A20299270297D4F48091E800877FB8
:104320008093E8008091A10280939A020E947C1EF3
:1043300080919A02811106C08091E30087FD02C03E
:1043400081E001C084E080939E020E94B61B8091B0
:10435000E80083FF0AC08091E800877F8093E8002F
:104360008091EB0080628093EB00AA960FB6F894E0
:10437000DEBF0FBECDBFDF91CF911F91089508958D
:10438000CF9380919E028823A1F0C091E900CF7065
:104390009091EC00892F817090FD80E8C82B1092DD
:1043A000E9008091E80083FD0E945F20CF70C093F8
:1043B000E900CF91089597FB072E16F4009407D0DB
:1043C00077FD09D00E94F52107FC05D03EF49095B9
:1043D00081959F4F0895709561957F4F0895EE0FD9
:1043E000FF1F0590F491E02D0994AA1BBB1B51E11E
:1043F00007C0AA1FBB1FA617B70710F0A61BB70B55
:10440000881F991F5A95A9F780959095BC01CD01F9
:104410000895FB01DC0104C08D910190801921F405
:1044200041505040C8F7881B990B0895F999FECF69
:1044300092BD81BDF89A992780B50895A8E1B0E0B2
:1044400042E050E00C944A22262FF999FECF92BD0B
:1044500081BDF89A019700B4021639F01FBA20BD49
:104460000FB6F894FA9AF99A0FBE08950396272F7B
:104470000E9425220E942422252F0E942522242FDB
:104480000C9425220196272F0E9425220C94242289
:10449000DC01CB01FC01F999FECF06C0F2BDE1BD04
:1044A000F89A319600B40D9241505040B8F70895F3
:0444B000F894FFCFAE
:1044B400C8001002280850011E0A1401FA1A1D1B14
:1044C400FE1A8D1B891BFD1A01E200E900EA00B502
:1044D40000B600B700CD008301CC008A019201949C
:1044E400012102230224022502260227022A02B302
:1044F40000B4006F007000818283E200E900EA00EA
:10450400B500B600B700CD008301CC008A0192014A
:1045140094012102230224022502260227022A02F0
:10452400B300B4006F007000818283F4F53534C6A3
:0C45340097669490919293F63332360013
:00000001FF
